:10000000D8000120710C00006D0C00006D0C000088
:100010006D0C00006D0C00006D0C00000000000075
:100020000000000000000000000000006D0C000057
:100030006D0C0000000000006D0C00006D0C000055
:100040006D0C00006D0C00006D0C00006D0C0000CC
:100050006D0C00006D0C00006D0C00006D0C0000BC
:100060006D0C00006D0C00006D0C00006D0C0000AC
:100070006D0C00006D0C00006D0C00006D0C00009C
:100080006D0C00006D0C00006D0C00006D0C00008C
:100090006D0C00006D0C00006D0C00006D0C00007C
:1000A0006D0C00006D0C00006D0C00006D0C00006C
:1000B0006D0C00006D0C00006D0C00006D0C00005C
:1000C0006D0C00006D0C00006D0C00006D0C00004C
:1000D0006D0C00006D0C00006D0C00006D0C00003C
:1000E0006D0C00006D0C000000000000000000001E
:1000F00000000000290500006D0C00006D0C0000E0
:100100006D0C00006D0C00006D0C00006D0C00000B
:100110006D0C00006D0C0000C90B0000350C0000D8
:100120003D0C0000450C00006D0C00006D0C000043
:100130006D0C00006D0C00006D0C00006D0C0000DB
:100140006D0C00006D0C00006D0C00006D0C0000CB
:100150006D0C00006D0C00006D0C00006D0C0000BB
:100160006D0C00006D0C00006D0C00006D0C0000AB
:100170006D0C00006D0C00006D0C00006D0C00009B
:100180006D0C00006D0C00006D0C00006D0C00008B
:100190006D0C00006D0C00006D0C00006D0C00007B
:1001A0006D0C00006D0C00006D0C00006D0C00006B
:1001B0006D0C00006D0C00006D0C00006D0C00005B
:1001C0006D0C00006D0C00006D0C00006D0C00004B
:1001D0006D0C00006D0C00006D0C00006D0C00003B
:1001E0006D0C00006D0C00006D0C0000A1130000F0
:1001F0006D0C00006D0C00006D0C00006D0C00001B
:100200006D0C00006D0C00006D0C00006D0C00000A
:100210006D0C00006D0C00006D0C00006D0C0000FA
:100220006D0C00006D0C00006D0C00006D0C0000EA
:100230006D0C00006D0C00006D0C00006D0C0000DA
:100240006D0C00006D0C00006D0C00006D0C0000CA
:100250006D0C00006D0C00006D0C00006D0C0000BA
:100260006D0C00000348044B834202D0034B03B1E2
:1002700018477047AC150000AC15000000000000E6
:100280000548064B1B1AD90F01EBA301491002D0F8
:10029000034B03B118477047AC150000AC150000C4
:1002A0000000000010B5064C237843B9FFF7DAFFD1
:1002B000044B13B10448AFF300800123237010BD39
:1002C0000000002000000000AC15000008B5044B41
:1002D0001BB104490448AFF30080BDE80840CFE7F4
:1002E0000000000004000020AC150000024A536822
:1002F0000342FCD1704700BF00280040174938B5C1
:100300004B68174D13F0010F10D10320A8470B784D
:100310009B0706D50B7803F0FD030B70A84702205E
:10032000A8470E4B01221A700320A8470B49012051
:10033000A8470B7803F0EF0300240B700320A847B5
:100340004C708C608C610C634C63CC610C620B78DC
:1003500043F002030B70A847204638BD0028004038
:10036000ED020000F0B505681DB90F4BBDE8F04087
:100370001847D1F808C02C460026C2F1010ED4E976
:100380000137934295BFDB1973449B1ADB199C45D7
:1003900007D92368264613B9044B3046E6E71C46C6
:1003A000EDE7A542E1D0F7E7710500009D050000EB
:1003B0002DE9F047D0E90465037E0136DA070446EB
:1003C00006611FD4037E9B071CD4DFF84480DFF84E
:1003D000449000F11407CDB16B68AA68F31A9342F8
:1003E00014D33846C0472B7C012B04D16E603246B3
:1003F00029463846C847D4F814A0EB6828469847E1
:100400005546E8E7237E43F002032376BDE8F087F4
:10041000A50500006503000038B50D46044610B17F
:10042000081E18BF01203B220549064B9847064B82
:10043000294620469847054B23600020206138BD9F
:100440004C140000B105000061120000B10300006F
:100450001FB50389ADF804304FF40043ADF8063002
:100460000391054B029201A91438144698470028BD
:1004700008BF204604B010BD5D0A00001FB5038907
:10048000ADF8043048F20103ADF806300391054B96
:10049000029201A9143814469847002808BF204644
:1004A00004B010BD5D0A000038B50446003818BF1E
:1004B0000120074B0D465E2206499847064B294608
:1004C0002046984718B9054BA361054B636138BDB9
:1004D000B105000063140000310A00007D04000033
:1004E000510400000A4A13889BB210B543F4A0637C
:1004F0001380084B9847084B9847084B9847084B80
:100500009847BDE81040074B40F6FF70184700BF02
:10051000004000410D0D0000B7050000F50500008A
:10052000B90500004D0C00000B4A937882B0DBB295
:100530000193019B990705D5084B1B6813B15068BF
:1005400002B01847019BDB0704D5044B5B680BB175
:10055000014AF4E702B07047000002411C0000208D
:10056000006800B970478842FAD101207047000046
:1005700038B5074B0446984780F001000D46054BFF
:1005800005493922C0B2984723682B60256038BDE1
:1005900061050000B10500007F14000003680B60D6
:1005A0000160704703680BB11A6802601846704713
:1005B00000B900BE704770470C4B0D4A5A63DA6BA6
:1005C00012F0060FFBD14FF402629A63022283F805
:1005D0003020064AD36B9807FCD4044B1A6CD10721
:1005E00002D41A6C9207F9D5704700BF0010004082
:1005F0004D0E0100014B01225A7170470008004066
:10060000C3690B42FCD170470268034B22F002021F
:1006100002600321184700BF010600000160014B82
:10062000032118470106000070B50C4D06460FCD9A
:1006300088B06C460FC495E80F0084E80F006A4646
:10064000002352F8041BB14202D1D8B208B070BDE9
:100650000133082BF5D10020F8E700BFB8140000E3
:1006600008B5034B984780002E3000F0FE0008BD0F
:10067000290600004109044A00F01F0001238340BD
:1006800042F82130704700BF00E100E0430906490D
:1006900000F01F0020330122824041F82320BFF3E5
:1006A0004F8FBFF36F8F704700E100E043090449AB
:1006B00000F01F0001226033824041F82320704780
:1006C00000E100E008B5074B9847032808D0002058
:1006D0000549064B40F2CE3298474FF0FF3008BD37
:1006E0000020FCE7290600009D140000B105000071
:1006F0004268034B42F4403242600421184700BF75
:10070000010600002DE9F0410D4614460421534A2C
:10071000D0F800809047438B15F0010F06469BB23E
:10072000174660D09D0716D501220276628892B2E4
:1007300042F480526280628803F0010522F48072E4
:100740001204C5F1FF25120C05F57F056280FC350A
:100750002846BDE8F08113F0040515D06368002B2E
:10076000C1BF63889BB243F48053638063881F04D6
:1007700001D53B4B9847638823F480731B041B0C03
:1007800063806FF00105E3E7638813F4806713D09B
:1007900027889047436AFF0907F0060703F4804360
:1007A0003B4343F0F10343629047638823F4806343
:1007B0001B041B0C6380CBE7656845B963881E0486
:1007C00001D5274B9847638823F48073F0E7D4F86A
:1007D000088018F8013B8362013D9047C4F8088007
:1007E00065600025B4E715F00205B1D06268002A03
:1007F00031D059072FD4013AC8F3C06362609AB967
:10080000ABB163881B0408D5736823F480737360ED
:1008100004213046B847124B9847638823F480730D
:100820001B041B0C63800BE0012A09D143B17368E0
:1008300043F48023736004213046B847002AE0D097
:1008400004213046B847A368B26A591CA1601A70E7
:1008500002233376C5E70223337692E701060000D0
:10086000F10600002DE9F0470C46214BDFF88CA083
:10087000204DDFF88C90064608469847E36913F050
:10088000010FC7B213D1182303FB07A303215B6A2F
:10089000204603F01C08A84723689B0703D5164B86
:1008A00098470221A84748F001012046C84718226E
:1008B00002FB07A220460121A847546A2146C847E7
:1008C000936A43600421A847D36AC360C4F30163F9
:1008D000B381436AC4F3406423F4804343EA84331E
:1008E0004362A847538EF3810020BDE8F08700BF24
:1008F000C50600000106000009060000B81400004B
:100900001D06000070B51A4B04469847022805D012
:100910001849194B40F26B2200209847E369174DA4
:10092000174E13F0010F0DD1164B032120469847A7
:1009300023689B0703D5144B98470221A84705213C
:100940002046B04720460121A8471049B0474FF440
:10095000403363601F21A8470D4BA3604FF611433E
:10096000A3810023A373184684F8303070BD00BF04
:10097000290600009D140000B105000001060000DA
:100980001D060000010600000906000004001040DA
:10099000020070002DE9F7430546003818BF01201A
:1009A000144B0C46CB2214499847144B20469847C9
:1009B0000646D8B9124BAC619C4208BF114BDFF818
:1009C000509008BF1D6020460F4BDFF848800F4F46
:1009D0009847002405462B19D8B20190C8470198C2
:1009E000C04701340198B847042CF4D1304603B015
:1009F000BDE8F083B10500009D140000050900006A
:100A0000002001412C000020610600007506000056
:100A10008D060000AD060000836999627047836906
:100A200001229A757047836902229A757047000007
:100A300070B504460D46064B064901204FF4A862E6
:100A40009847256129462046034BBDE8704018476A
:100A5000B10500009D140000650800002DE9F04775
:100A60000446DFF85C9107690E464FF4BF625149B6
:100A70000120C84720694F49003840F2F95218BF99
:100A80000120C847301E18BF01204A4940F2FA52DF
:100A9000C8476388D8057AD47388DFF828819BB269
:100AA00043F48073738096E807007B6843F4807397
:100AB00084E807007B6004213846C04725693D492A
:100AC000D5F800A040F2CD520120C8476368012B41
:100AD0006B6839D11AF0006F36D043F480236B6015
:100AE00004212846C047238859054FEA43022ED5E2
:100AF0006388DB0741BF63889BB243F480636380F4
:100B00000421C04722F001026B6A5205520D03F422
:100B100080431A4342F400426A62C04722694FF49C
:100B20008033117E013BC9B201D08807F9D0284635
:100B30002246214DA847D0B1638823F480731B045B
:100B40001B0C6380BDE8F08723F48023C7E7B4F86B
:100B500002900421C0471FFA89F96B6AD2B209F0EA
:100B6000010942EA090203F480431A43D4E7638887
:100B7000DA05E7D522694FF48033117E013BC9B213
:100B800008D08807F9D022463846A847EFE76FF02B
:100B90000500D7E773881B0402D5084B38469847F1
:100BA000638823F480731B041B0C63806FF00400C4
:100BB000C8E700BF9D14000005070000F106000013
:100BC000B105000001060000194B186810B58469D2
:100BD000237EDA0708D5A37DDB0705D5012323751E
:100BE0000368BDE810401847237E990706D5A37D0A
:100BF0009A0703D5022323758368F2E7237E5B07F8
:100C00000CD5638B03F0370313B1FF23638310BD4F
:100C1000A16A4368BDE81040C9B21847237EDB09CA
:100C2000F5D080232376C3689847638B9BB2EDE7AA
:100C30002C000020004B1847C90B0000004B184740
:100C4000C90B0000004B1847C90B0000C30707D5AC
:100C5000044B054A1A6243F6FD7259681142FCD1F1
:100C6000704700BF001C004007010100FEE70000C4
:100C700018491948814210B50AD0184BDA1C121ACB
:100C800022F00302C41EA34238BF0022144B98472F
:100C9000144B1548DA1C121AC11E22F003029942A5
:100CA00088BF0022114B00219847114A114B22F0B6
:100CB0007F029A60D3F8882042F47002C3F888203B
:100CC000BFF34F8FBFF36F8F0B4B98470B4B98477A
:100CD000FEE700BFAC15000000000020000000206F
:100CE00021140000D8000020000000203D14000066
:100CF0000000000000ED00E0D9130000010D00002D
:100D000008B5014B9847FEE701120000064B42F27E
:100D10008E329A8200229A75DA75DA6902F47C5270
:100D2000DA6101221A747047001400404309DB01A4
:100D300003F1824330B503F5004300F01F041D1991
:100D400003EB540395F8402002F0FE0242F001024A
:100D500085F8402093F8302010F0010FC9B21BBF76
:100D600002F00F0242EA011202F0F002D2B20ABF10
:100D7000114383F8302083F8301030BD054B4022FA
:100D8000C3F89020044A536943F480635361034BD2
:100D9000184700BF001C004000080040051100007B
:100DA000064B4022C3F8DC204322C3F88C20044ABF
:100DB000936943F400739361704700BF001C0040C7
:100DC0000008004010B5054C05493920A0472346CE
:100DD0000449BDE810403820184700BF2D0D000021
:100DE000030039000300380013B5074B0749084CCE
:100DF0009847084A002300931023D018A047064BB9
:100E000002B0BDE810401847A10D000000200141CC
:100E10004910000030000020C50D000070B50B4CDB
:100E20000B4D94F856300B4903F0FB0384F8563011
:100E30001620A84794F85730074903F0FB0384F8BD
:100E4000573017202B46BDE87040184700800041FE
:100E50002D0D00000200160002001700064B402274
:100E6000C3F8E0204322C3F88C20044A936943F47A
:100E700080639361704700BF001C00400008004081
:100E800010B5054B054906489847064B9847BDE8FD
:100E90001040054B184700BF5D0E000000400141A7
:100EA00090000020A90400001D0E000010B50D4B9D
:100EB00098470D4B98470D4B98470D4B98470D4A57
:100EC000536943F4804353610B4B4022C3F8A42081
:100ED0000A4B9847BDE810400246094909480A4BA9
:100EE000184700BFE50400007D0D0000E90D00007B
:100EF000810E000000080040001C00409D1300000F
:100F000000380040B0000020190400000023836274
:100F1000C3690BB108381847704700238362436ADE
:100F20000BB108381847704770B50446054BA0F15F
:100F300008052C309847236A1BB12846BDE870404D
:100F4000184770BDA111000070B50E461546044645
:100F500018B1D9B1101E18BF01200F4B0F4940F234
:100F60003B129847B4F84420B4F84C309A420FD161
:100F70000023A4F844300123236304F10800084B44
:100F8000A664A4F84C509847284670BD0846E4E78C
:100F90006FF01B00F9E700BFB1050000011500006C
:100FA0001F0A0000838FB0F844209A4210B504460F
:100FB0000AD0026C591C8187D15C044B9847044BC2
:100FC0002046BDE810401847024BFAE7190A000016
:100FD0001F0A0000270A00002DE9F7430E461746B6
:100FE000044618B1E9B1101E18BF01201049114B79
:100FF000DFF850904FF4AC72984734340E4B01A890
:1010000098470E4B204698470D4B804601A89847BD
:101010000025A84501D0BD4205D1284603B0BDE852
:10102000F0830846E2E771192046C8470135F0E72A
:1010300001150000B1050000BD130000E111000022
:10104000CB13000061110000F8B50D4616461F468F
:10105000044620B109B312B3181E18BF012012496B
:10106000124B3A229847124B3A46314604F134006B
:101070009847B0B90F4B294604F10800984758B972
:101080000D4B63600D4B23600D4BA3600D4BE36074
:101090000D4B23610D4B6361F8BD0846DFE7104639
:1010A000DDE76FF00C00F7E701150000B105000067
:1010B0002511000095090000D90F0000490F00001C
:1010C000A50F0000290F00000D0F00001B0F0000EE
:1010D0000B4930B44D68012200239A4201D230BC42
:1010E0007047D4186408FAD1854204D10B68002BEC
:1010F000F5D030BC18472CBFFF220123EDE700BF1D
:10110000CC000020044B054800224FF0FF31C3E91A
:101110000021034B184700BFCC000020D110000075
:10112000FD02000070B50E461446054618B189B19F
:10113000101E18BF01200849084B28229847631E3B
:1011400013EA040003BFC5E90130E8602E606FF0C8
:101150000C0070BD0846EEE71E150000B10500004A
:1011600038B50D46044610B1081E18BF01200A4BC1
:101170000A4940229847D4E902329A4209D062686B
:1011800013402268D35C2B70A3680133A360002056
:1011900038BD6FF00900FBE7B10500001E15000027
:1011A00038B504460D460C4B0C4951220120984796
:1011B000E368626813402268D554D4E90121E368EA
:1011C000591A914288BF9A1A03F1010388BFA2609D
:1011D000E360002038BD00BFB10500001E1500000F
:1011E00010B50549054B0446672201209847D4E90C
:1011F0000230C01A10BD00BF1E150000B10500006E
:10120000004B1847AD0E000003690B42FCD170473C
:1012100070B5104D06460FCD88B06C460FC495E8EA
:101220000F0084E80F006A46002052F8041BB14208
:1012300002D130B908B070BD01300828F5D10020C6
:10124000F8E700200449054B4FF49E7298474FF091
:10125000FF30EFE75815000042150000B10500000F
:101260002DE9F843454B814608460C469847444BC8
:101270004449C9F80C408D228046012098472369D3
:10128000414A13F0010F11D10321204690472368F2
:101290009B0706D5236823F00203236090470221B1
:1012A000904701232360032120469047374F1425A0
:1012B00005FB08750121204690476E6A26600321D0
:1012C000904795F82A30E37306F00C062B8DE380E7
:1012D000082E4FF0010323733AD1EB6AE361C0217A
:1012E000904700232362904701236372284B9C425E
:1012F00004BF284BC3F80090142303FB0873B3F911
:101300002230002B0DDB5A09012103F01F03994005
:1013100002F12003204A42F82310BFF34F8FBFF39E
:101320006F8F142303FB0870B0F92230002B0CDB05
:1013300003F01F015B099B0003F1604303F5614368
:1013400001228A40C3F880211A600020BDE8F8839A
:101350002EB9AB8DA383C0219047E683C3E7042E4B
:10136000C2D195F82C302377C021904700236377B2
:10137000904795F82B30E3762021B4E71112000056
:10138000B1050000421500000912000058150000C8
:1013900000380040D400002000E100E00020704749
:1013A000054B1868C3689A7AD20703D501229A724E
:1013B00003681847704700BFD4000020EFF3108384
:1013C000036072B6BFF35F8F7047BFF35F8F036830
:1013D00083F310887047000070B50D4D0D4C641BF1
:1013E000A4100026A64209D10B4D0C4C00F0CEF8FB
:1013F000641BA4100026A64205D170BD55F8043B1D
:1014000098470136EEE755F8043B98470136F2E776
:101410009815000098150000981500009C15000014
:101420000A44914200F1FF3300D1704710B511F822
:10143000014B03F8014F9142F9D110BD024403461C
:10144000934200D1704703F8011BF9E72E2E2F6855
:10145000616C2F7372632F68616C5F74696D657264
:101460002E63002E2E2F68616C2F7372632F6861BC
:101470006C5F6932635F6D5F73796E632E63002EFC
:101480002E2F68616C2F7574696C732F7372632FC4
:101490007574696C735F6C6973742E63002E2E2FE4
:1014A00068706C2F736572636F6D2F68706C5F73FB
:1014B0006572636F6D2E63000030004000340040A1
:1014C00000200141004001410000004300040043AE
:1014D00000080043000C004303000000140020003B
:1014E00000010000FF0000000000D70000042707F3
:1014F00000000000000000000000000000000000EC
:10150000002E2E2F68616C2F7372632F68616C5FE1
:1015100075736172745F6173796E632E63002E2E32
:101520002F68616C2F7574696C732F7372632F75DC
:1015300074696C735F72696E676275666665722E38
:1015400063002E2E2F68706C2F74632F68706C5F91
:1015500074632E630000000000380040003C00402F
:1015600000A0014100C001410014004200180042E7
:10157000001400430018004300006B000803000043
:1015800000000000973A000000000000F8B500BF1E
:10159000F8BC08BC9E467047CD020000F8B500BFFD
:0C15A000F8BC08BC9E467047A502000085
:00000001FF
